:10000000830100308A0004288301282B831290008A
:10001000911B112811088A001008900A0319910AEF
:1000200082008313111883171008900A84000008B7
:100030000800483465346C346C346F343A342034FE
:0200400000348A
:1006140083128510013083121B2B83128C0004304B
:100624008D00FA3083121B238D0B132B8C0B112B93
:10063400080083128C0004308D0053308E008E0B22
:10064400212B8D0B1F2B8C0B1D2B08008316850172
:100654000130860083128501860183120A23193032
:100664008C0000308D0038234B23362B422B0D0891
:1006740091000C088C0A03198D0A062083128A2320
:1006840083120D0891000C08062000380319080095
:10069400392B83128C01061C4D2B29308D008D0BB8
:1006A400512B061C0C1421308D008D0B572B061C6E
:1006B4008C1421308D008D0B5D2B061C0C15213004
:1006C4008D008D0B632B061C8C1521308D008D0B3A
:1006D400692B061C0C1621308D008D0B6F2B061C0C
:1006E4008C1621308D008D0B752B061C0C172130B8
:1006F4008D008D0B7B2B061C8C1721308D008D0BF0
:10070400812B21308D008D0B852B0C0883128A2BB5
:1007140083128E008E09851421308F008F0B902B4D
:100724000E0C031C972B8514982B85100310831231
:100734008E0C21308F008F0B9D2B0E0C031CA42BD1
:100744008514A52B8510031083128E0C21308F0085
:100754008F0BAA2B0E0C031CB12B8514B22B851006
:10076400031083128E0C21308F008F0BB72B0E0CCD
:10077400031CBE2B8514BF2B8510031083128E0C13
:1007840021308F008F0BC42B0E0C031CCB2B851434
:10079400CC2B8510031083128E0C21308F008F0B0D
:1007A400D12B0E0C031CD82B8514D92B85100310C8
:1007B40083128E0C21308F008F0BDE2B0E0C031C4A
:1007C400E52B8514E62B8510031083128E0C213043
:1007D4008F008F0BEB2B0E0C031CF22B8514F32BC9
:1007E4008510031083128E0C21308F008F0BF82B91
:0C07F400851021308F008F0BFD2B0800BA
:02400E00F93F78
:00000001FF
